:10000000830100308A001628A00003088301B10094
:1000100021088100A10803190F28043085060B115F
:10002000831231088300A00E200E090021308400C5
:100030002C30282083010330B000FE30AF002C307C
:1000400084002D302C208301AF2B04068001840A0C
:100050000406031D25280034AD0037208000840AE3
:1000600004082D06031900342D288312AF00B01B9D
:10007000402830088A002F08AF0A0319B00A82000E
:100080008313301883172F08AF0A84000008080074
:10009000FF3496347C340C3400340C347C340C340F
:1000A00000340C346C340C3463340C344F3410345E
:1000B000003406347C340C3400340C347C340C347E
:1000C00000340C346C340C3463340C344F3410343E
:1000D0000034063463340C3400340C3463340C3490
:1000E00000340C3439340C342D340C3413341034C3
:1000F0000034063439340C3400340C342D340C34D0
:1001000000340C3413341834003418348B3418345D
:10011000983418349E340C3498340C348B3418349E
:100120009E341834A9341834B2341834A93418342D
:100130009E341834B2341834BF341834B7340C3405
:10014000BF340C34B2341834A9341834B2341834EF
:10015000003418348B341834983418349E340C34EA
:1001600098340C348B3418349E341834A934183431
:10017000B2341834A9341834C63410340034063478
:10018000C634103400340634BF341834B2340C345E
:10019000BF340C34B234103400340634B23410346A
:1001A00000340634C634183400341834C6341034DD
:1001B000003406348B34103400340634C634103422
:1001C000003406348B34103400340634C634103412
:1001D000003406348B34103400340634C634103402
:1001E000003406348B3410340034063400341834B0
:1001F000C6341834BF34103400340634BF341034DD
:1002000000340634B2341834BF341834C6341834C9
:1002100000341834C6341034003406348B341034AF
:1002200000340634C6341034003406348B341034B1
:1002300000340634C6341034003406348B341034A1
:1002400000340634C6341034003406348B34103491
:100250000034063400341834C6341834BF34103433
:1002600000340634BF34103400340634B234183449
:10027000A9341834B234183400341834BF34183464
:1002800000341834BF34183400341834BF341834F0
:1002900000341834BF34183400341834BF340C34EC
:1002A00000340C34BF340C3400340C34B7340C3408
:1002B000B2340C34A934103400340634BF340C3456
:1002C00000340C34BF340C3400340C34B7340C34E8
:1002D000B2340C34A9341034003406349E3418344B
:1002E000A9341834B2340C3400340C34B7340C3420
:1002F000B2340C34A93418349E341834BF34183452
:1003000000341834BF340C3400340C34BF340C3493
:1003100000340C34B7340C34B2340C34A9341034F7
:1003200000340634BF340C3400340C34BF340C3485
:1003300000340C34B7340C34B2340C34A9341034D7
:1003400000340634B2340C3400340C34B2340C347F
:1003500000340C349E340C3498340C348B34103408
:10036000003406349E340C3400340C3498340C348D
:1003700000340C348B3418340034183400343034E6
:04038000FF34003412
:1006AE000230A600602B851014308223851414307E
:1006BE0082238312A603260F5A2B8B138B12051C33
:1006CE00662BFF30831685000000373095009601AB
:1006DE00960A0B108B158B13630000008B110B10F9
:1006EE008B16F93085009501950A8B1783128510AC
:1006FE00051808007F2BA701A801AB00A22B2C0820
:10070E00AD00AE010310AD0DAE0D0310AD0DAE0D6F
:10071E000310AD0DAE0D2D08A9002E08AA00FF3056
:10072E008312A907031CAA032A082904031D962B6A
:10073E00A70A0319A80A83122B08AD00AE012808D8
:10074E002E06031DAC2B27082D0603190800862B39
:10075E00A201A301FF238316900007308312990094
:10076E0083169F01FD3085008312850181018B1751
:10077E000B17A1010230831681008B1683125723AB
:10078E0083122308003EB0002208483E0318B00A28
:10079E003520A4002308AE002208AD000130AD07BD
:1007AE000318AE0A2E08003EB0002D08483E03186E
:1007BE00B00A3520A500240FEF2BA508031DEA2B48
:1007CE00A201A301C52B83122508AC000230FA2B1F
:1007DE0083120518F42B572383122408A100250831
:1007EE00822302308506A2070318A30AC72B64349E
:02400E008431FB
:00000001FF
